 can

 Timestamp is 4da293cb (Mon Apr 11 17:38:19 2011)

 Preferred load address is 10000000

 Start         Length     Name                   Class
 0001:00000000 00000004H .CRT$XCA                CODE
 0001:00000004 00000004H .CRT$XCZ                CODE
 0001:00000008 00000004H .CRT$XIA                CODE
 0001:0000000c 00000004H .CRT$XIZ                CODE
 0001:00000010 00000004H .CRT$XPA                CODE
 0001:00000014 00000004H .CRT$XPZ                CODE
 0001:00000018 00000004H .CRT$XTA                CODE
 0001:0000001c 00000004H .CRT$XTZ                CODE
 0001:00000020 0000002cH .rdata                  CODE
 0001:0000004c 00000020H .rdata$debug            CODE
 0001:0000006c 00001a2cH .text                   CODE
 0001:00001a98 00000048H .xdata                  CODE
 0001:00001ae0 0000003cH .idata$2                CODE
 0001:00001b1c 00000014H .idata$3                CODE
 0001:00001b30 000000a8H .idata$4                CODE
 0001:00001bd8 000000a6H .idata$6                CODE
 0001:00001c80 00000102H .edata                  CODE
 0002:00000000 000000a8H .idata$5                DATA
 0002:000000a8 00000008H .data                   DATA
 0002:000000b0 00000010H .bss                    DATA
 0003:00000000 00000168H .pdata                  DATA

  Address         Publics by Value              Rva+Base       Lib:Object

 0000:00000000       ___safe_se_handler_count   00000000     <absolute>
 0000:00000000       ___safe_se_handler_table   00000000     <absolute>
 0001:00000000       __xc_a                     10001000     corelib0:crt0init.obj
 0001:00000004       __xc_z                     10001004     corelib0:crt0init.obj
 0001:00000008       __xi_a                     10001008     corelib0:crt0init.obj
 0001:0000000c       __xi_z                     1000100c     corelib0:crt0init.obj
 0001:00000010       __xp_a                     10001010     corelib0:crt0init.obj
 0001:00000014       __xp_z                     10001014     corelib0:crt0init.obj
 0001:00000018       __xt_a                     10001018     corelib0:crt0init.obj
 0001:0000001c       __xt_z                     1000101c     corelib0:crt0init.obj
 0001:0000003c       ??_C@_1M@EENNDIOJ@?$AAI?$AAn?$AAd?$AAe?$AAx?$AA?$AA@ 1000103c     can_common_topaz_v1:can_io.obj
 0001:00000048       ??_7?$Buffer_t@VDuplicateTraits_t@detail@marshal@ce@@@detail@marshal@ce@@6B@ 10001048     can_common_topaz_v1:can_io.obj
 0001:0000006c       CANConfigureGPIO           1000106c f   bspcan.obj
 0001:000002ac       BSPCANClockConfig          100012ac f   bspcan.obj
 0001:000002fc       BSPCANConfigureGPIO        100012fc f   bspcan.obj
 0001:00000328       BSPGetCANBaseRegAddr       10001328 f   bspcan.obj
 0001:00000350       BSPGetCANIRQ               10001350 f   bspcan.obj
 0001:00000370       BSPSetCanPowerEnable       10001370 f   bspcan.obj
 0001:000003a0       ?Unmarshal@MarshalledBuffer_t@@QAAJXZ 100013a0 f i can_common_topaz_v1:can_io.obj
 0001:000003f8       ?CAN_Init@@YAKPBG@Z        100013f8 f   can_common_topaz_v1:can_io.obj
 0001:0000047c       ?CAN_Open@@YAKKKK@Z        1000147c f   can_common_topaz_v1:can_io.obj
 0001:00000480       ?CAN_Close@@YAHK@Z         10001480 f   can_common_topaz_v1:can_io.obj
 0001:00000488       ?CAN_PowerDown@@YAXK@Z     10001488 f   can_common_topaz_v1:can_io.obj
 0001:0000048c       ?CAN_PowerUp@@YAXXZ        1000148c f   can_common_topaz_v1:can_io.obj
 0001:00000490       ?CAN_Read@@YAKKPAXK@Z      10001490 f   can_common_topaz_v1:can_io.obj
 0001:00000498       ?CAN_Write@@YAKKPBXK@Z     10001498 f   can_common_topaz_v1:can_io.obj
 0001:000004a0       ?CAN_Seek@@YAKKJG@Z        100014a0 f   can_common_topaz_v1:can_io.obj
 0001:000004a8       ?Free@?$Buffer_t@VDuplicateTraits_t@detail@marshal@ce@@@detail@marshal@ce@@QAAJXZ 100014a8 f i can_common_topaz_v1:can_io.obj
 0001:000004ec       ?Marshal@MarshalledBuffer_t@@QAAJPAXKKHH@Z 100014ec f i can_common_topaz_v1:can_io.obj
 0001:0000057c       ?CAN_Deinit@@YAHK@Z        1000157c f   can_common_topaz_v1:can_io.obj
 0001:000005a0       ??0?$Buffer_t@VDuplicateTraits_t@detail@marshal@ce@@@detail@marshal@ce@@QAA@PAXKK@Z 100015a0 f i can_common_topaz_v1:can_io.obj
 0001:000005f0       ??_E?$Buffer_t@VDuplicateTraits_t@detail@marshal@ce@@@detail@marshal@ce@@UAAPAXI@Z 100015f0 f i can_common_topaz_v1:can_io.obj
 0001:000005f0       ??_G?$Buffer_t@VDuplicateTraits_t@detail@marshal@ce@@@detail@marshal@ce@@UAAPAXI@Z 100015f0 f i can_common_topaz_v1:can_io.obj
 0001:00000628       ?CAN_IOControl@@YAHKKPAEK0KPAK@Z 10001628 f   can_common_topaz_v1:can_io.obj
 0001:00000c40       ??1CANClass@@QAA@XZ        10001c40 f   can_common_topaz_v1:canclass.obj
 0001:00000cfc       ?CANEnableTLPRIOMode@CANClass@@QAAHH@Z 10001cfc f   can_common_topaz_v1:canclass.obj
 0001:00000d20       ?CANReset@CANClass@@QAAHXZ 10001d20 f   can_common_topaz_v1:canclass.obj
 0001:00000d40       ?CANPowerHandler@CANClass@@QAAHH@Z 10001d40 f   can_common_topaz_v1:canclass.obj
 0001:00000d7c       ?CANSetMode@CANClass@@QAAXKW4_CAN_MODE@@@Z 10001d7c f   can_common_topaz_v1:canclass.obj
 0001:00000dc8       ?WritePacket@CANClass@@QAAHPAUCAN_PACKET@@H@Z 10001dc8 f   can_common_topaz_v1:canclass.obj
 0001:00000ef8       ?ReadPacket@CANClass@@QAAHPAUCAN_PACKET@@H@Z 10001ef8 f   can_common_topaz_v1:canclass.obj
 0001:00001004       ?ProcessPackets@CANClass@@QAAHQAUCAN_PACKET@@H@Z 10002004 f   can_common_topaz_v1:canclass.obj
 0001:00001098       ?CANInterruptHandler@CANClass@@AAAXI@Z 10002098 f   can_common_topaz_v1:canclass.obj
 0001:000012d8       ?CANIST@CANClass@@CAXPAX@Z 100022d8 f   can_common_topaz_v1:canclass.obj
 0001:000012e8       ??0CANClass@@QAA@I@Z       100022e8 f   can_common_topaz_v1:canclass.obj
 0001:0000153c       CeCloseCallerBuffer        1000253c f   coredll:COREDLL.dll
 0001:0000154c       CeFreeAsynchronousBuffer   1000254c f   coredll:COREDLL.dll
 0001:0000155c       CeAllocDuplicateBuffer     1000255c f   coredll:COREDLL.dll
 0001:0000156c       CeFreeDuplicateBuffer      1000256c f   coredll:COREDLL.dll
 0001:0000157c       RegCloseKey                1000257c f   coredll:COREDLL.dll
 0001:0000158c       RegQueryValueExW           1000258c f   coredll:COREDLL.dll
 0001:0000159c       OpenDeviceKey              1000259c f   coredll:COREDLL.dll
 0001:000015ac       DisableThreadLibraryCalls  100025ac f   coredll:COREDLL.dll
 0001:000015bc       CeAllocAsynchronousBuffer  100025bc f   coredll:COREDLL.dll
 0001:000015cc       CeOpenCallerBuffer         100025cc f   coredll:COREDLL.dll
 0001:000015dc       EventModify                100025dc f   coredll:COREDLL.dll
 0001:000015ec       KernelIoControl            100025ec f   coredll:COREDLL.dll
 0001:000015fc       CloseHandle                100025fc f   coredll:COREDLL.dll
 0001:0000160c       InterruptDisable           1000260c f   coredll:COREDLL.dll
 0001:0000161c       InterruptDone              1000261c f   coredll:COREDLL.dll
 0001:0000162c       WaitForSingleObject        1000262c f   coredll:COREDLL.dll
 0001:0000163c       CeSetThreadPriority        1000263c f   coredll:COREDLL.dll
 0001:0000164c       LeaveCriticalSection       1000264c f   coredll:COREDLL.dll
 0001:0000165c       EnterCriticalSection       1000265c f   coredll:COREDLL.dll
 0001:0000166c       InitializeCriticalSection  1000266c f   coredll:COREDLL.dll
 0001:0000167c       CreateThread               1000267c f   coredll:COREDLL.dll
 0001:0000168c       InterruptInitialize        1000268c f   coredll:COREDLL.dll
 0001:0000169c       CreateEventW               1000269c f   coredll:COREDLL.dll
 0001:000016ac       MmUnmapIoSpace             100026ac f   ceddk:CEDDK.dll
 0001:000016bc       MmMapIoSpace               100026bc f   ceddk:CEDDK.dll
 0001:000016cc       DDKIomuxSelectInput        100026cc f   cspddk:CSPDDK.dll
 0001:000016dc       DDKGpioWriteDataPin        100026dc f   cspddk:CSPDDK.dll
 0001:000016ec       DDKGpioSetConfig           100026ec f   cspddk:CSPDDK.dll
 0001:000016fc       DDKIomuxSetPadConfig       100026fc f   cspddk:CSPDDK.dll
 0001:0000170c       DDKIomuxSetPinMux          1000270c f   cspddk:CSPDDK.dll
 0001:0000171c       DDKClockSetGatingMode      1000271c f   cspddk:CSPDDK.dll
 0001:0000172c       DllMain                    1000272c f   corelib0:dllmain.obj
 0001:00001838       _DllMainCRTStartup         10002838 f   corelib0:pegdmain.obj
 0001:00001924       _cexit                     10002924 f   corelib0:cexit.obj
 0001:00001934       _initterm                  10002934 f   corelib0:crt0dat.obj
 0001:00001960       _cinit                     10002960 f   corelib0:crt0dat.obj
 0001:000019c0       __security_init_cookie     100029c0 f   corelib0:seccinit.obj
 0001:00001a0c       __crt_ExitProcess          10002a0c f   corelib0:exitproc_proxy.obj
 0001:00001a18       ??2@YAPAXI@Z               10002a18 f   corelib1:COREDLL.dll
 0001:00001a28       ??3@YAXPAX@Z               10002a28 f   corelib1:COREDLL.dll
 0001:00001a38       __C_specific_handler       10002a38 f   corelib1:COREDLL.dll
 0001:00001a48       memset                     10002a48 f   corelib1:COREDLL.dll
 0001:00001a58       _XcptFilter                10002a58 f   corelib1:COREDLL.dll
 0001:00001a68       free                       10002a68 f   corelib1:COREDLL.dll
 0001:00001a78       __security_gen_cookie2     10002a78 f   corelib1:COREDLL.dll
 0001:00001a88       TerminateProcess           10002a88 f   coredll:COREDLL.dll
 0001:00001ae0       __IMPORT_DESCRIPTOR_COREDLL 10002ae0     coredll:COREDLL.dll
 0001:00001af4       __IMPORT_DESCRIPTOR_CEDDK  10002af4     ceddk:CEDDK.dll
 0001:00001b08       __IMPORT_DESCRIPTOR_CSPDDK 10002b08     cspddk:CSPDDK.dll
 0001:00001b1c       __NULL_IMPORT_DESCRIPTOR   10002b1c     coredll:COREDLL.dll
 0002:00000000       __imp_MmUnmapIoSpace       10003000     ceddk:CEDDK.dll
 0002:00000004       __imp_MmMapIoSpace         10003004     ceddk:CEDDK.dll
 0002:00000008       \177CEDDK_NULL_THUNK_DATA  10003008     ceddk:CEDDK.dll
 0002:0000000c       __imp_CeFreeDuplicateBuffer 1000300c     coredll:COREDLL.dll
 0002:00000010       __imp_RegCloseKey          10003010     coredll:COREDLL.dll
 0002:00000014       __imp_RegQueryValueExW     10003014     coredll:COREDLL.dll
 0002:00000018       __imp_OpenDeviceKey        10003018     coredll:COREDLL.dll
 0002:0000001c       __imp_DisableThreadLibraryCalls 1000301c     coredll:COREDLL.dll
 0002:00000020       __imp_CeAllocAsynchronousBuffer 10003020     coredll:COREDLL.dll
 0002:00000024       __imp_CeOpenCallerBuffer   10003024     coredll:COREDLL.dll
 0002:00000028       __imp_EventModify          10003028     coredll:COREDLL.dll
 0002:0000002c       __imp_KernelIoControl      1000302c     coredll:COREDLL.dll
 0002:00000030       __imp_CloseHandle          10003030     coredll:COREDLL.dll
 0002:00000034       __imp_CeAllocDuplicateBuffer 10003034     coredll:COREDLL.dll
 0002:00000038       __imp_InterruptDone        10003038     coredll:COREDLL.dll
 0002:0000003c       __imp_WaitForSingleObject  1000303c     coredll:COREDLL.dll
 0002:00000040       __imp_CeSetThreadPriority  10003040     coredll:COREDLL.dll
 0002:00000044       __imp_LeaveCriticalSection 10003044     coredll:COREDLL.dll
 0002:00000048       __imp_EnterCriticalSection 10003048     coredll:COREDLL.dll
 0002:0000004c       __imp_InitializeCriticalSection 1000304c     coredll:COREDLL.dll
 0002:00000050       __imp_CreateThread         10003050     coredll:COREDLL.dll
 0002:00000054       __imp_InterruptInitialize  10003054     coredll:COREDLL.dll
 0002:00000058       __imp_CreateEventW         10003058     coredll:COREDLL.dll
 0002:0000005c       __imp_CeFreeAsynchronousBuffer 1000305c     coredll:COREDLL.dll
 0002:00000060       __imp_InterruptDisable     10003060     coredll:COREDLL.dll
 0002:00000064       __imp_CeCloseCallerBuffer  10003064     coredll:COREDLL.dll
 0002:00000068       __imp___security_gen_cookie2 10003068     corelib1:COREDLL.dll
 0002:0000006c       __imp_free                 1000306c     corelib1:COREDLL.dll
 0002:00000070       __imp__XcptFilter          10003070     corelib1:COREDLL.dll
 0002:00000074       __imp_memset               10003074     corelib1:COREDLL.dll
 0002:00000078       __imp_??2@YAPAXI@Z         10003078     corelib1:COREDLL.dll
 0002:0000007c       __imp_??3@YAXPAX@Z         1000307c     corelib1:COREDLL.dll
 0002:00000080       __imp___C_specific_handler 10003080     corelib1:COREDLL.dll
 0002:00000084       __imp_TerminateProcess     10003084     coredll:COREDLL.dll
 0002:00000088       \177COREDLL_NULL_THUNK_DATA 10003088     coredll:COREDLL.dll
 0002:0000008c       __imp_DDKIomuxSetPinMux    1000308c     cspddk:CSPDDK.dll
 0002:00000090       __imp_DDKIomuxSetPadConfig 10003090     cspddk:CSPDDK.dll
 0002:00000094       __imp_DDKGpioSetConfig     10003094     cspddk:CSPDDK.dll
 0002:00000098       __imp_DDKGpioWriteDataPin  10003098     cspddk:CSPDDK.dll
 0002:0000009c       __imp_DDKIomuxSelectInput  1000309c     cspddk:CSPDDK.dll
 0002:000000a0       __imp_DDKClockSetGatingMode 100030a0     cspddk:CSPDDK.dll
 0002:000000a4       \177CSPDDK_NULL_THUNK_DATA 100030a4     cspddk:CSPDDK.dll
 0002:000000a8       __security_cookie          100030a8     corelib0:seccinit.obj
 0002:000000ac       __security_cookie_complement 100030ac     corelib0:seccinit.obj
 0002:000000b0       _exitflag                  100030b0     corelib0:cexit.obj
 0002:000000b4       __onexitend                100030b4     <common>
 0002:000000b8       __onexitbegin              100030b8     <common>
 0002:000000bc       _pRawDllMain               100030bc     <common>

 entry point at        0001:00001838

 Static symbols

 0001:00001748       _DllMainCRTStartupHelper   10002748 f   corelib0:pegdmain.obj
 0001:00001864       doexit                     10002864 f   corelib0:cexit.obj
